:10000000830100308A000428203084004B300F2008
:1000100083010A128A110E2D04068001840A040647
:10002000031D0C28003483120313CB00CC1B2128A2
:100030004C1B29284C088A004B08CB0A0319CC0A10
:10004000820083134C1883174B08CB0A84000008E6
:10005000080083014C0C1F39831203178F00031310
:100060004B0C03178D0083168C170C140000000036
:1000700083120C0883014B184328831203178C1B2F
:1000800003140E0D83017F390800D229A018A51E84
:1000900034182C32531032293D10B012641A41002A
:1000A00030373D10B012641A2016EE20A018A51E9D
:1000B00034180032EE202019A51E34182C324110BD
:1000C0002021A01EB012581A47004928B127201A33
:0600D000652AF43900105E
:1007900083010800F0000030711870070310F00D9D
:1007A0000310F10CF10803190800CC2BF401F5013A
:1007B0000310F30CF20C031CE42B7008F40771080F
:1007C0000318710AF5070310F00DF10D7208730498
:1007D00003190034D82B8301B500831611141118A6
:1007E000EF2B911283128C11403093008C1DF62B4D
:1007F0008C11350893008C1DFB2B8C1183169114E2
:100800009118002C83128C11413093008C1D062C02
:100810008C1183169115141C0B2C83121308B60728
:10082000831691161116111A132C11151119162C65
:100830008312360808008301BD00831611141118B5
:100840001F2C911283128C11403093008C1D262C8A
:100850008C113D0893008C1D2B2C8C118316911448
:100860009118302C83128C11413093008C1D362C42
:100870008C1183169115141C3B2C83121308BF0096
:10088000BE0183161116111A432C9115141C462C07
:1008900083121308BE070318BF0A83169116111698
:1008A000111A502C11151119532C83123F08F10005
:1008B0003E08F00008008301BE00831611141118D1
:1008C0005F2C83128C11403093008C1D652C8C1191
:1008D0003E0893008C1D6A2C8C113D0893008C1DE2
:1008E0006F2C8C11831611151119742C83120800AA
:1008F0008301BD008316111411187C2C83128C11F6
:10090000C63093008C1D822C8C1193018C1D862C7B
:100910008C113D088400831380080319972C3D082F
:10092000840000089300BD0A8C19882C942C83162F
:1009300011151119992C831208008301BD0083162B
:1009400011141118A12C83128C11C63093008C1D28
:10095000A72C8C1193018C1DAB2C8C1102309300B1
:100960008C1DB02C8C113D0893008C1DB52C8C1166
:10097000831611151119BA2C83120800831603135C
:1009800011141118C12C83128C11C63093008C1DC8
:10099000C72C8C1193018C1DCB2C8C110C30930027
:1009A0008C1DD02C8C11043093008C1DD52C8C11F7
:1009B000831611151119DA2C83120800FE308301F9
:1009C000860083168600FF30870083128700803000
:1009D00083169400383083129400831691013230CC
:1009E00093008312BD01BE01BF01C001BD0A0319FE
:1009F000BE0A0319BF0A0319C00A00304002031DD2
:100A00000B2D04303F02031D0B2D93303E02031DBE
:100A10000B2DE0303D0203180800F62CDE24BE2426
:100A200005309D24C930BE004030BF0020300A127E
:100A30008A11BB250A128A1120307824BD01BD0A13
:100A400000305B248030BD0003305B240D30BD00DE
:100A500000305B240330BD0000305B2401301B24D8
:100A60007008B5007108B6000430BD0000305B248A
:100A700001301B247008B7007108B80015309D24A0
:100A80009F30BE004030BF003708BB003808BC00B4
:100A90003508B9003608BA003930BD0020300A12D6
:100AA0008A11BB250A128A11203078240530BD0036
:100AB00000305B2401301B247008B5007108B600BB
:100AC00004301B247008B7007108B80029309D2439
:100AD000B430BE004030BF003708BB003808BC004F
:100AE0003508B9003608BA003930BD0020300A1286
:100AF0008A11BB250A128A11203078240A30BD00E1
:100B000000305B248F018E01313090000C100C1CE2
:100B1000872D101001301B247008B5007108B60035
:100B20000B30BD0000305B248F018E01313090000E
:100B30000C100C1C992D101001301B247008B700EC
:100B40007108B8003D309D248A30BE004030BF009F
:100B50003708BB003808BC003508B9003608BA00B1
:100B60003930BD0020300A128A11BB250A128A11C1
:100B7000203078242A2D8301C600C4013D08C1001D
:100B8000AE2F4508253A031D9F2FFF30C200C30139
:100B9000C001612FC6080319D12D460884008313B4
:100BA0008001440808000230C10741028400831319
:100BB00000089D2FC00AE02D0830C207FE30C20792
:100BC0000230C1074102840083130008C700840A71
:100BD0000008C8004018C81FF42DC709C809C70A73
:100BE0000319C80AC303F52DC0010B30C207420820
:100BF000F200F3014808F1004708F0000A128A11D8
:100C0000C6277008C5004208F200F3014708F0004B
:100C10004808F1000A128A11C6270A128A117408BC
:100C2000C7007508C800C901C90ACA014A084802B4
:100C3000031D1C2E49084702031C412E4208F200E6
:100C4000F3014908F0004A08F1000A128A11D6237C
:100C50000A128A117408C9007508CA00C303162E47
:100C6000C40AC60803193B2E4608840083132030AB
:100C70008000C60A412E20300A128A11C8230A12A7
:100C80008A11C3034308803A7F3E0318302E401C6C
:100C9000562EC40AC6080319522E46088400831330
:100CA0002D30912E2D300A128A11C8234208F200ED
:100CB000F3014908F0004A08F1000A128A11C62718
:100CC0000A128A117408C9007508CA004904031978
:100CD000972E4A08F3004908F2004808F100470837
:100CE000F0000A128A11C6277408F0007508F10096
:100CF0004208F200F3010A128A11C6270A128A1169
:100D00007008C300803A763E031C882E0730C30764
:100D1000C40AC6080319942E4608840083134308A6
:100D2000303E8000C60A562E4308303E532E0A300D
:100D30004502031C9D2E0730C507C40AC6080319C7
:100D4000A72E4608840083134508303EA72F450888
:100D5000303EAB2FC40AC6080319B52E46088400DE
:100D6000831320308000C60ABB2E20300A128A115D
:100D7000C8230A128A11C3034308803A7E3E03182F
:100D8000AA2E0230C1074102840083130008C50067
:100D90009F2F0230C1074102840083130008C9005D
:100DA000840A0008CA00C50145084907CB004A0863
:100DB000CC004B080318CC0A0A128A1113200A121D
:100DC0008A1100380319E62EC50AD42E42084502BE
:100DD0000318EC2E4508C2004208C31B232FFF3A1C
:100DE0004307031C232FC40AC6080319FE2E460816
:100DF0008400831320308000C60A042F20300A129A
:100E00008A11C8230A128A11C303EC2E4A08CC00A7
:100E100049080A128A1113200A128A11C500C90A48
:100E20000319CA0AC40AC60803191D2F46088400FC
:100E3000831345088000C60A232F45080A128A1129
:100E4000C8230A128A11C203420F062FAE2F3F0891
:100E5000CC003E080A128A1113200A128A112A3A7B
:100E6000031D392F0230C10741028400831300089B
:100E70005D2F3F08CC003E080A128A111320D03E95
:100E8000C200BE0A0319BF0A3F08CC003E080A127E
:100E90008A1113200A128A11C50030304502031C42
:100EA000612F3A3045020318612F0A30F1004208E1
:100EB0000A128A11CA234507D03EC200BE0A03198E
:100EC000BF0A3F08CC003E08BE0A0319BF0A0A1237
:100ED0008A1113200A128A11C500003A0319CA2D7B
:100EE0002A3A0319D32D043A0319272F763A031906
:100EF000DC2D3B3A0319BC2E073A0319DA2D0B3AC5
:100F00000319DE2D1C3A0319C92E063A0319E02DE8
:100F10000D3A0319DC2D30304502031C9F2F3A3067
:100F2000450203189F2F0A30F10043080A128A1164
:100F3000CA230A128A114507D03EC300612FC40A92
:100F4000C6080319AA2F46088400831345088000A9
:100F5000C60AAE2F45080A128A11C8233F08CC00E2
:100F60003E08BE0A0319BF0A0A128A1113200A1288
:100F70008A11C500C508031DC12DC6080319C42F59
:100F8000460884008313800144080800F601F40138
:100F9000F50172087304031DD02FF001F101003434
:100FA0001F30F6040310F60AF20DF30D031CD32FC5
:100FB000F30CF20C73087102031DE02F720870022B
:100FC000031CE82F7208F0027308031C730AF10275
:100FD000F40DF50DF60BF61AD82FF61FF42FF409C1
:100FE000F40A0319F503F5097408F2007508F30013
:100FF000761F0034F009F00A0319F103F1090034F7
:02400E00323B43
:00000001FF
